:10000000A42A82004F347C2957345B345F345D343A
:1000100072297C294D345134553459347B34FF34A2
:100020007C297C2906293F347C290229DF34FD34D0
:100030007C297C297C299D34BD34BF34DD34FB34DC
:100040007C297C2999349B34BB34DB34F734F93474
:100050007C297C297F349734B934D734D934F534AA
:100060007C297C2993349534B534B734D534F334B2
:100070007C297C297C299134B334D334F134EF3496
:100080007C297C298F34B134D134CF34EB34ED3436
:100090007C297C298D348B34AF34AD34CD34E934B4
:1000A0007C297C297C29AB347C29CB34E7347C291E
:1000B0007C2967293D347734C9347C29A9347C29CB
:1000C0007C297C299F347C297C297C297C297D34CE
:1000D0007C297C29C5347C29A53485347C297C295C
:1000E0007C29E1348734C334A334A1348334753498
:1000F0005F297C294334C1346B34453481347529FC
:100100007C297C297C297C29533423297C297C293E
:100110007C297C297C297C297C297C297C297C29B7
:100120007C297C2909297C297C2900297C297C2996
:100130007C297C297C297C297C297C297C297C2997
:100140000C297C297C297C297C297C297C297C29F7
:1001500012297C297C297C297C297C297C297C29E1
:1001600018297C297C297C297C297C297C297C29CB
:100170007C297C297C297C297C297C297C297C2957
:100180007C297C297C297C297C297C297C297C2947
:100190007C297C297C2947347C297C297C297C2961
:1001A0007C297C297C297C297C297C297C297C2927
:1001B0007C297C297C2979347C297C297C297C290F
:1001C0007C297C297C297C297C297C297C297C2907
:1001D0007C297C2937297C2961342D297C297C299B
:1001E00063347929733465347C29633467347C291A
:1001F0007C297C297C2941297C2923294B297C299C
:100200009E1F7C291A141A1A1A1039349E1E0E29A0
:1002100037349E1E142935349E1E37349A141A1A08
:100220009A1033349E1E35341A151A1A1A113134A5
:100230009D1C7C291A1E00343330B6219130EB21ED
:100240003230B62100341D1F7C291A1E0034313093
:10025000B621CD30EB21303021291D1D7C291A1EFD
:1002600000343D30B6216130EB213C3021299D1D09
:100270007C291A1E00343D30B6216330EB213C301E
:1002800021299D1E7C291A1E00343D30B62165307F
:10029000EB213C3021291D1E7C291A1E00343D30E3
:1002A000B6216730EB213C3021291E1C7C291A1E07
:1002B00000343930B6219930EB21383021291E1E07
:1002C0004B341A1E003402309B06972100349E1DC9
:1002D0007C291A1E003404309B0697213B301B1DDD
:1002E000FE3921291E197C2941349E187C299A1235
:1002F00000349D1F7C29413494092E30B6211E30D4
:1003000091001A1A11119A1991109A1E911111083F
:10031000B62114089100910D11081E39B621940ED2
:10032000940D14081E39212901301B069B00ED3065
:10033000F2212B220508F8391B0485001B08F22145
:100340002B2AA3210030962125309100AA21910B60
:10035000A6290800FF3092006400920BAD29080026
:1003600090000F020319080010088F0090000A3057
:10037000A52108309100A300901B8515901F8511C1
:100380000A30AB2105120A30AB2105160A30AB2129
:10039000900D910BBC298316851583129101920152
:1003A000851DDA296400910BD029920BD0291A1BE4
:1003B0000800E6291A1B080091018519E129910B13
:1003C000DD2985158316851183120800E121910A24
:1003D000A30BC02908009700B6211708FE39B621E3
:1003E0001708080094009501861400000610831673
:1003F00086100000061083120830910083168614C0
:1004000083128618012A14180614141C0610940C62
:100410000318950A861C0A2A910B012A86180E2AAF
:1004200015180610151C0614861C142A8618162A80
:100430000614861C192A83160614831286181E2A8F
:10044000861C202A0830AB21861083168610831262
:100450001430AB21080096011A169A1186148316DF
:1004600086148312861C3D2A6400061B322A9A1EBB
:10047000322AA11FE32BA1138C2A861C3D2A0830A7
:1004800091008618412A940C06189417061C9413A0
:10049000861C482A910B412A86184C2A861C4E2A13
:1004A0008618502A861C522A88221430AB2116083E
:1004B00003195C2A96032E2AE130140203197B2AC1
:1004C000E030140203197F2AF03014020319812A44
:1004D0009A1D732A1230140203192B2A5930140260
:1004E00003192B2A080083301402031D08009A15F3
:1004F0000330940008005521073096002C2A9A15E5
:100500002E2A1A122E2A86148316861483120800A5
:10051000861083168610862A0F30B6211A170F30E0
:10052000B6211630930085199C2A910B932A920BC1
:10053000932A9421930B932A051283160611831292
:10054000FF30A521A11FD52B202307309A008F0152
:1005500010303C239D003D239E003D239F003D2302
:10056000A0003D23A100061CB32AFF30F221073072
:10057000A121F3309F21FF309F21F0309F210230D5
:10058000F2211E1BC52AA11FD52B0230B621023035
:10059000B6219A161A08073903198C2A9A1EEF2ACF
:1005A0002B221A19E02A1E1BDA2ACA239A1BDA2ADE
:1005B000A1138C2A9A18E02A073014020319452B3C
:1005C000941FE42A7C21CA2A140A9A19803E012029
:1005D000003E0319CA2A1A1EFE39B021CA2A061281
:1005E0009C01A20191014030920883226400861C84
:1005F000002B910BF62A920BF62A882294211C2BB1
:100600008023003E031D1C2B3D2314020319A20A64
:100610005A301402031D182B22081C02031DEF2A56
:10062000FF3094007C211B1097219A160616CA2AC7
:1006300010301C020319EF2A1C0894007C21F22AB6
:1006400083121830850018308600831681138501C7
:10065000C73086008312080088001C0889009C0AA5
:100660008316081555308900AA3089008814081EA1
:10067000372B8801831208009C001C0889009C0A03
:10068000831608148312080808001A123330EB216D
:100690003130EB214330EB2180239C2316301402B0
:1006A0000319572B1E30140203196F2BA42A9C0127
:1006B00080236630140203196B2B9C2314082C230F
:1006C0005A30140203194A2B0F301C02031D582BF9
:1006D0005A3094005D2B1C08031D9C03582B1030CE
:1006E0009C008023A2239800980E9C238023A223A1
:1006F00018042C239C2314301C02031D712B4A2B3D
:100700002B22941B952B1A1E952B9A19952B910130
:100710005930982358309823113098231230982359
:10072000143098231108031900349A1E0134802BC9
:1007300014020319910A0800140A0120003E03194B
:100740000800EB29910192011630C1231E30C1230C
:100750002630C1232530C1232E30C1233630C1239A
:100760003D30C1233E30C1234630C1231C30C1235C
:100770003230C1232130C1232330C1232430C1238F
:100780002B30910A14020319C72B12080800110814
:10079000920008009A171A08F7381F02031D080074
:1007A0002008140203199A130800A11314309C00A6
:1007B00021082C2386118616EA232B221A1EDD2BF4
:1007C000CA239A1BDD2BA11714309C0021082C236F
:0E07D000EA23A42AED23061FEA2B8030A52978
:084000000000020001000000B5
:02400E00F73F7A
:104200001C003A00430034001C005A00FF00FF006D
:10421000FF00FF00FF00FF00FF00FF00FF00FF00A6
:0A422000FF00FF00F7007600FF002A
:00000001FF
